:100000000C9479040C9472340C94B1040C94B104E3
:100010000C94B1040C94B1040C94B1040C94B1048C
:100020000C94B1040C94B1040C948D2B0C94492BBA
:100030000C94E02C0C94B1040C94B1040C94B10415
:100040000C94B1040C94B1040C94B1040C94B1045C
:100050000C94B1040C94BC2C0C94B1040C94B10419
:100060000C94B1040C94B1040C94B1040C94B1043C
:100070000C94B1040C94B1040C94B1040C94B1042C
:100080000C94B1040C94B1040C94B1040C94B1041C
:100090000C94B1040C94B1040C94B1040C94B1040C
:1000A0000C94B1040C94B1040C94B1040631FF0912
:1000B00074A1010975150026FF00952075088102BD
:1000C0000976150026FF00952075089102C00501EC
:1000D0000980A101850319012AB700150126B7007F
:1000E000950175108100C0050C0901A10185041955
:1000F000012AA002150126A002950175108100C0F9
:100100000660FF0961A1010962150026FF00952024
:10011000750881020963150026FF00952075089176
:1001200002C005010906A101050719E029E715002C
:100130002501950875018102950175088101050762
:10014000190029FF150026FF009506750881000596
:10015000081901290595057501910295017503910D
:1001600001C00000000000000000000000000000CE
:10017000000000000000000000000000000000007F
:100180000000000000007E0F00D4FFFFFFC700004A
:10019000007800000000000000002A2B280000006A
:1001A0000000000000000000000000000029000026
:1001B00000002C1E3420212224342627252E362D03
:1001C0003738271E1F202122232425263333362E9D
:1001D00037381F0405060708090A0B0C0D0E0F100F
:1001E0001112131415161718191A1B1C1D2F313054
:1001F000232D350405060708090A0B0C0D0E0F10F8
:100200001112131415161718191A1B1C1D2F313033
:10021000354C726762206D617472697820746F6703
:10022000676C65205B25735D3A207267625F6D6164
:10023000747269785F636F6E6669672E656E61625E
:100240006C65203D2025750A0044454255473A20FB
:1002500064697361626C65642E0A004445425547C7
:100260003A20656E61626C65642E0A004F6E65739C
:10027000686F743A206163746976653A2025640A70
:10028000000A002530325820006B6579626F617278
:10029000645F7265706F72743A20005461726765B2
:1002A0007420636F6E6E65637465640D0A0054613B
:1002B0007267657420646973636F6E6E65637465DD
:1002C000642C207468726F74746C696E6720636F3D
:1002D0006E6E656374696F6E20617474656D7074A1
:1002E000730D0A004661696C656420746F2065783F
:1002F00065637574652025730A007267625F6D61BE
:10030000747269785F636F6E6669672E666C616789
:1003100073203D2025640A007267625F6D6174720C
:1003200069785F636F6E6669672E737065656420B8
:100330003D2025640A007267625F6D61747269789E
:100340005F636F6E6669672E6873762E76203D2038
:1003500025640A007267625F6D61747269785F6319
:100360006F6E6669672E6873762E73203D20256454
:100370000A007267625F6D61747269785F636F6EA5
:100380006669672E6873762E68203D2025640A0012
:100390007267625F6D61747269785F636F6E6669C0
:1003A000672E6D6F6465203D2025640A00726762C8
:1003B0005F6D61747269785F636F6E6669672E65E1
:1003C0006E61626C65203D2025640A007267625F81
:1003D0006D61747269785F636F6E66696720454509
:1003E00050524F4D0A007267625F6D617472697896
:1003F0005F696E69745F6472697665727320726793
:10040000625F6D61747269785F636F6E6669672E93
:100410006D6F6465203D20302E2057726974652011
:1004200064656661756C742076616C7565732074A3
:100430006F20454550524F4D2E0A007267625F6D26
:1004400061747269785F696E69745F6472697665F8
:100450007273206565636F6E666967206973206ECD
:100460006F7420656E61626C65642E0A005B735D5B
:10047000000A0025303862003A200025303258004A
:100480000A722F632030313233343536370A000A8E
:100490000025303258006C65645F7461736B3A20DC
:1004A0000000010101010101010101020202020239
:1004B000020202020303030303030303040404040C
:1004C00004040405050505050606060606070707D4
:1004D000070708080808090909090A0A0A0B0B0B8B
:1004E0000C0C0C0D0D0D0E0E0E0F0F0F1010111128
:1004F00011121213131414151516161717181819AC
:10050000191A1A1B1B1C1D1D1E1E1F202021222212
:10051000232424252626272829292A2B2C2D2D2E55
:100520002F30313232333435363738393A3B3C3D6F
:100530003E3F404142434445464748494A4C4D4E60
:100540004F50515354555658595A5B5D5E5F616226
:1005500064656668696B6C6D6F7072737577787AB5
:100560007B7D7E8082838587888A8C8E8F91939510
:1005700096989A9C9EA0A2A3A5A7A9ABADAFB1B334
:10058000B5B7BABCBEC0C2C4C6C9CBCDCFD1D4D614
:10059000D8DBDDDFE2E4E7E9EBEEF0F3F5F8FAFDB6
:1005A000FF6565636F6E6669675F7570646174652A
:1005B0005F7267625F6D61747269785F64656661BE
:1005C000756C740A00726762206D617472697820BC
:1005D0006D6F6465205B25735D3A2025750A007296
:1005E0006762206D61747269782073657420687326
:1005F00076205B25735D3A2025752C25752C257595
:100600000A00726762206D61747269782073657484
:10061000207370656564205B25735D3A2025750A3B
:10062000004E004B00AA00A9004D004A00AC00ABF0
:1006300000C55CC65CC75CC85CCB5CCC5CC95CCAF2
:100640005C29001E001F002000210022002B001446
:10065000001A00080015001700E00004001600074B
:100660000009000A00E1001D001B0006001900053A
:100670000000000000E300105F28004A002A002765
:100680000026002500240023004C00130012000C5B
:100690000018001C00340033000F000E000D000B8A
:1006A00000E500380037003600100011000000009F
:1006B00000E600115F2C004D0035021E021F0220D3
:1006C0000221022202005C1E001F002000210022E5
:1006D000004C00010050004F0052002F00C05C0190
:1006E000000100010051002F020000000001000184
:1006F000004C0026022A002702260225022402239B
:100700000201002700260025002400230031022ECC
:10071000025E005D005C00300001002D005B005AAD
:10072000005900300200000000620001004C002768
:100730000245003A003B003C003D003E00C25C1E0A
:10074000021F02200221022202C35CAC00AB00A9FE
:10075000004B002D02A800AD00AE00AA004E002DF7
:1007600000000000000100010001002602440043D7
:10077000004200410040003F000100270226022500
:1007800002240223023100C95CC75CC55C4A002E0A
:10079000000100CA5CC85CC65C4D002E020000006F
:1007A0000001000100010001000100010001000141
:1007B0000001000100010001000100010001000131
:1007C0000001000100010001000100010001000121
:1007D0000001000100010001000000000001000113
:1007E0000001000100010001000100010001000101
:1007F00000010001000100010001000100010001F1
:1008000000010001000100010001000100010001E0
:1008100000010001000000000001000100010001D2
:10082000005B435D005B445D005B535D005B575DB7
:10083000005B525D0009027B00040100A0FA09047C
:100840000000010301010009211101000122400003
:1008500007058103080001090401000203000000EC
:100860000921110100012222000705820320000155
:100870000705030320000109040200010300000032
:100880000921110100012232000705840320000123
:1008900009040300020300000009211101000122E4
:1008A000220007058503200001070505032000013C
:1008B000120100020000000810CB5663100601026E
:1008C00000011A0349007200690073002000520001
:1008D000650076002E0020003600610000000E0347
:1008E0004B0065006500620069006F0000000403B2
:1008F000090411241FBECFEFDAE0DEBFCDBF04B67E
:1009000003FE18C080912B0590912C05A0912D0518
:10091000B0912E058730904BA740B04B59F4109200
:100920002B0510922C0510922D0510922E05E0E05B
:10093000F8E3099512E0A0E0B1E0EEEFFDE602C0B9
:1009400005900D92AE3FB107D9F725E0AEEFB2E0CA
:1009500001C01D92AB32B207E1F70E94072D0C9443
:10096000AF360C940000FF93EF93E091FE02F091FC
:10097000FF02309709F00995EF91FF910895FC016E
:100980008591803011F0EFDFFBCF0895FF27E0E283
:1009900030E247FF0CC0419597FF09C0EDE260953A
:1009A000709580959095611D711D811D911D27FF8A
:1009B00002C0219530E350E2AA27660F771F881FF7
:1009C000991FAA1FA41710F0A41B63955A95A9F7A5
:1009D000AA3008F0A95FA05DAF93F395611571058A
:1009E0008105910541F7ED3211F4EF93F395F2177C
:1009F00018F43F93F395FBCF8F91B5DFFA95E1F7AC
:100A00000895E991F9918591803021F0853219F0AE
:100A1000AADFF9CF089520E0E89455915532C1F34B
:100A2000503311F4689455915A3348F4505390F36D
:100A3000220F022E220F220F200D250FF4CF0EF4CD
:100A4000219589919991533619F3533729F15335EB
:100A500059F1BC0188279927E8945C3621F48991E3
:100A6000999168945591543639F446EF7EF077FFAA
:100A70000DC08FEF9FEF0AC055374AE039F0583567
:100A800040E121F0523642E009F00895FF93EF93E0
:100A90007DDFEF91FF91B7CFFF93EF93FC01819141
:100AA0008030B9F360DFFBCFFF93EF9368DFF1CFC6
:100AB000DF93CF93CDB7DEB72596A3DFCF91DF913C
:100AC0000895E8EDF0E080818E7F80831092E2004F
:100AD0001092DA001092E100A0EEB0E08C918160FB
:100AE0008C9380818F77808319BCA7EDB0E08C91C7
:100AF0008E7F8C9380818F7E80831092DD04089599
:100B00002091E4003091E50095E6A9012091EC00E8
:100B1000822F817020FF06C08091E80080FF06C010
:100B200080E008952091E80022FD1AC08091EA0437
:100B3000882389F0853089F08091EB0085FD0FC016
:100B40002091E4003091E50042175307F9F29150EB
:100B5000E1F684E0089582E0089583E0089581E05D
:100B60000895EF92FF920F931F93CF937C018B0117
:100B70000E948005C82F811117C08091E80085FD73
:100B80000BC08091E8008E778093E8000E9480057A
:100B9000882399F3C82F08C0F70181917F018093C2
:100BA000F1000150110949F78C2FCF911F910F913E
:100BB000FF90EF9008958091EC0487FF13C080911F
:100BC000E80082FF06C08091E8008B778093E80000
:100BD00004C08091EA048111F2CF08958091EA0463
:100BE0008823D9F38091E80080FFF8CF8091E80056
:100BF0008E77ECCF982F9093E900242F762F50E03A
:100C0000891731F07091EC002091ED005091F000C7
:100C100021FD07C09F5F973071F78093E90081E065
:100C200008953091EB003E7F3093EB003091ED0062
:100C30003D7F3093ED003091EB0031603093EB005D
:100C40007093EC002093ED005093F0002091EE00A3
:100C500027FDE0CF80E00895B0E0A0E0E2E3F6E019
:100C60000C949835C8EDD0E088818F7E8883E7EDBD
:100C7000F0E080818160808384E082BF81E08093A6
:100C8000DD0488818E7F888302EE10E0F8011082F7
:100C90001092DA0081EEC82ED12CF60110828881E4
:100CA0008F77888388818068888388818F7D888317
:100CB00019BC1092EA041092EB041092E90410920D
:100CC000E80490EEE92EF12CF70180818B7F808380
:100CD00088818160888342E060E080E00E94FA05BC
:100CE000F60180818E7F8083F8018081816080831E
:100CF000808188608083F70180818E7F80838881F6
:100D000080618883CDB7DEB7E8E00C94B435FC0190
:100D10008091F2049091F30486179707A0F0611573
:100D2000710529F49091E8009E779093E80090E097
:100D30006115710551F4911108C08091E80082FF9E
:100D400034C080E00895BC01F2CF8091EA0488238A
:100D5000C1F18530C1F18091E80083FD30C0809100
:100D6000E80082FDEACF8091E80080FFE1CF80912A
:100D7000F3002091F200382F6115710519F0283029
:100D8000310558F091E02830310509F090E02091CC
:100D9000E8002E772093E800CBCF81918093F1007B
:100DA000615071092F5F3F4FE7CF8091EA0488239C
:100DB00041F0853041F08091E80083FFBECF81E0B3
:100DC000089582E0089583E008950895089580913C
:100DD000DF0408959C014FB7F8948091D30490915B
:100DE000D404A091D504B091D6044FBF821B930BBD
:100DF00008952FB7F8946091D3047091D404809132
:100E0000D5049091D6042FBF08952FB7F894809100
:100E1000D3049091D404A091D504B091D6042FBFEF
:100E200008959C01FC0132969FEF80E041914617A6
:100E300051F09F3F19F4411101C0982F8F5F863008
:100E4000A9F79F3F09F40895290F311D97FD3A95A1
:100E5000F901628308952091D0043091D1042817BC
:100E6000390771F09093D1048093D004E091CE04BF
:100E7000F091CF04309721F00084F185E02D0995A1
:100E800008952091CC043091CD042817390771F0D2
:100E90009093CD048093CC04E091CE04F091CF04E4
:100EA000309721F00680F781E02D09950895FC0127
:100EB000680F791F8FEF91E32191822728E030E0BE
:100EC00087FF09C0880F892721503109C9F7E61724
:100ED000F70791F70895880FF7CFFA01811101C044
:100EE000FB010995089580934B018091250583703E
:100EF00080934A010E941D1483E080934C01089561
:100F0000EF92FF920F939701201B31092F3F31057C
:100F100019F010F02FEF30E02095382F320F08F441
:100F20003FEF832F0F91FF90EF900895EF92FF9284
:100F30000F939701201B31092F3F310519F010F055
:100F40002FEF30E0322F3095482F430F08F44FEF4A
:100F5000842F620F0F91FF90EF900895EF92FF9210
:100F60000F93972F093438F4B701601B71096F3F55
:100F7000710519F010F06FEF70E0485F5F4F41317D
:100F8000510540F0A901485F5F4F4131510510F014
:100F90006FEF70E06095482F460F08F44FEF842FF5
:100FA00037FF02C02D5F3F4F359527953595279523
:100FB00060912605620F792F0F91FF90EF900895B1
:100FC000EF92FF920F931F930E0D1F2D111DF9012C
:100FD00037FF03C0F195E195F10924E0EE0FFF1F03
:100FE0002A95E1F7EF3FF10519F014F0EFEFF0E08B
:100FF0009A0157FF03C031952195310994E0220FE2
:10100000331F9A95E1F72E173F070CF4F901E00F13
:10101000F11FEF3FF10519F010F0EFEFF0E0E09570
:10102000282F3E2F230F08F42FEF822F1F910F91AF
:10103000FF90EF900895EF92FF920F93970195E044
:10104000099F200D311D11242F3F310519F010F09B
:101050002FEF30E02095382F320F08F43FEF832F29
:101060000F91FF90EF90089522E8241B08F420E0F0
:10107000620F08954095282F429F412D1124842FFF
:1010800008950F931F9310E0F801EE0FFF1FE25D2C
:10109000FD4F9081905797FD9195000F111FF8011A
:1010A000EE50FE4F05AD0052110B2003F001219FC1
:1010B000F00D112408E310E0091B110997FD1395A9
:1010C00040039001419F300D1124E20FF31F9F0157
:1010D000220F331F2E0F3F1F37FF02C021583F4FF3
:1010E000220F232F221F330B620F1F910F910895A0
:1010F0000F931F93522F10E0F801EE0FFF1FEE50D9
:10110000FE4FA5ADA052BB0B9D015203F001539FB2
:10111000F00D1124000F111FD801A25DBD4F0C91DD
:101120000057110B40039001419F300D11242E0FE9
:101130003F1F37FF02C0215C3F4F96E03595279552
:101140009A95E1F7620F1F910F9108950F931F93E6
:10115000522F10E0F801EE0FFF1FEE50FE4FA5AD2D
:10116000A052BB0B9D015203F001539FF00D1124BF
:10117000000F111FD801A25DBD4F0C910057110B3C
:1011800040039001419F300D11242E0F3F1F37FF68
:1011900002C021583F4F220F232F221F330B620F13
:1011A0001F910F910895EF920F93972F23E0029FC5
:1011B000B0011124759567956E0D792F0F91EF9001
:1011C0000895322F50E0FA01EE0FFF1FEE50FE4F50
:1011D00095AD905297FD9195440F551FFA01E25D30
:1011E000FD4F2081231B330B290F311D97FD3A95AD
:1011F000620F0895E42FF0E0EE0FFF1FEE50FE4F58
:1012000065AD621B0895E42FF0E0EE0FFF1FE25D75
:10121000FD4F6081621B0895622F0895E42FF0E076
:10122000EE0FFF1FE25DFD4F408134EE439F412DE5
:101230001124E82FF0E050E0445E5F4FDA01A21B7A
:10124000B1099D01B7FF03C031952195310993E0A4
:10125000220F331F9A95E1F7AF01421B530B9A01FE
:1012600057FD20E0582F259F212D1124822F08950E
:10127000E42FF0E0EE0FFF1FE25DFD4F408134EE02
:10128000439F412D1124E72FF0E050E0445E5F4F73
:10129000DA01A21BB1099D01B7FF03C03195219569
:1012A000310993E0220F331F9A95E1F7AF01421BFA
:1012B000530B9A0157FD20E0279F212D1124722FF7
:1012C00008950E94630B0895FF920F931F93CF938D
:1012D000DF93182F062FF42ED0E0C0E02F2D402FE3
:1012E000612FCE010E9461092196C434D105B1F766
:1012F000CDB7DEB7E5E00C94B735FC019B01009754
:1013000029F480E077FF2BC080E80895AC0197FFB7
:1013100004C044275527481B590BB901640F751F9A
:1013200037FD10C0241B350BC901A5E0880F991F9C
:10133000AA95E1F70E94E53580E2861BF7FF0FC012
:1013400081950895CB0165E0880F991F6A95E1F7B3
:10135000BA01621B730B0E94E53580E6EECF08955B
:10136000EF920F93CF93DF93D72FC82FC9010E1998
:10137000BA010E947D09602F681B7D2F8C2FDF91A1
:10138000CF910F91EF9008950F93CF93DF93D72FC5
:10139000C82FC901BA010E947D09682F600F7D2FF7
:1013A0008C2FDF91CF910F910895EF920F931F93A0
:1013B000CF93DF93D62FC72F182FC9010E19010F16
:1013C000BA010E947D09081B202F219F212D112485
:1013D000822F6D2F7C2FDF91CF911F910F91EF9076
:1013E0000895EF920F931F93CF93DF93D62F172F6C
:1013F000C82FC9010E19070FBA010E947D09702F6D
:10140000781B719F712D11246D2F8C2FDF91CF913F
:101410001F910F91EF9008950F931F93CF93DF9338
:10142000D62FC72F182FC901212F201B022FBA0139
:101430000E947D09982F990F990F891B800F282FE3
:10144000219F212D1124822F6D2F7C2FDF91CF9191
:101450001F910F9108950F931F93CF93DF93D62F72
:10146000172FC82FC901272F201B022FBA010E9456
:101470007D09982F990F990F782F791B700F719F05
:10148000712D11246D2F8C2FDF91CF911F910F9112
:101490000895E82F86FDE0952E2F2F7086FD2F5F93
:1014A000E695E695E695E670F0E0EA52FE4F91810A
:1014B000929F902D212D112492959F702295207F2F
:1014C000922B2081920F87FD919580E8890F0895D6
:1014D000AC018230910508F408959FEF413E8EE102
:1014E000580740F49A0195E0369527959A95E1F7CB
:1014F00098E0920F61E0E62FE90FFF27FF1F9F01A1
:1015000035952795822F229FF001239FF00DF00D36
:1015100011244E175F0738F49FEF920F961758F774
:101520008FEF860F08952F3FE9F361E0620FF6CF4A
:101530000F93CF93DF93D72FC82F47FD419588E3B3
:1015400090E0841B910947FD9395889FB001899F86
:10155000700D700D1124229FC001239F900D900DDE
:101560001124860F971F0E94680A982F990F890FE0
:10157000682F600F7D2F8C2FDF91CF910F910895F1
:1015800030E020E0869F212D969F200D311D1124F3
:10159000C9010895AF92BF92CF92DF92FF920F934D
:1015A0001F93CF93DF93362F472FE82FF0E0EF55AF
:1015B000FB4F71110FC0E4918E2F2E2F6E2F722FC3
:1015C000DF91CF911F910F91FF90DF90CF90BF904F
:1015D000AF900895C72FD0E02491F22E022F10E093
:1015E00056E0659FC0011124EFEFF0E0BF010E94BB
:1015F000D135832F90E0880F991F35E5369FD001B4
:10160000379FB00D11248A1B9B0B982F990F980FB1
:101610006F01CC1ADD0AC09ED001C19EB00DD09ED4
:10162000B00D11248B2F499FA0011124452F552760
:101630006F01C41AD50AC09EA001C19E500DD09E54
:10164000500D11245F01A91AB108AC9E6001AD9E36
:10165000D00CBC9ED00C1124CD2CDD24EC19FD093E
:10166000E09FE001E19FD00DF09FD00D1124ED2F00
:1016700062307105A1F050F46115710509F49ECF37
:101680006130710581F0EB2F852F98CF64307105A3
:1016900069F080F06630710509F490CFF4CFE22F45
:1016A0002B2F8D2F8BCFE22F252F88CFEB2F822F43
:1016B0002D2F84CF2B2F8F2DE52F80CF89B185FB48
:1016C000882780F90895FF920F931F93CF93DF939C
:1016D000EC01F62E042F122F0E945E0B81110FC019
:1016E000C232D1057CF0A297FE01EE0FFF1FEC0F76
:1016F000FD1FE050FC4FF1820083128303C0C23211
:10170000D10594F3CDB7DEB7E5E00C94B735CF93B0
:10171000C82F0E945E0B882329F081E0C23228F096
:1017200080E003C081E0C434D8F7CF910895A8E0E9
:10173000B0E0EDE9FBE00C948E35282E7C836B83C2
:1017400020914E018EE0289F802D11248D83825F91
:101750008983853410F034E439830E945E0B88233A
:1017600029F08981833210F092E299830E945E0B06
:10177000811105C0ED81E23210F4F2E2FD83209187
:10178000F8042A839D81892F90E098878F83880FA2
:10179000991FFC01EE50FE4F6F01822D90E09C01DD
:1017A0002F5F3F4F3E832D8389819F81981730F0B3
:1017B0000E94870B2896E2E10C94AA35EF81F88508
:1017C000EA54FD4F808190914F018923F9F03090C8
:1017D0002605409027058D819E8188509B4F3C01B6
:1017E000522C10E0FA815F16D8F020912805129F44
:1017F000112D1124632D742D812F0E94CA0A462FAA
:10180000282F672F8F8198850E9461092F81388545
:101810002F5F3F4F38872F8332E0C30ED11CC4CFD8
:10182000F30181913F01F601A4ACA81ABB0885AC75
:10183000F3018781881A9908AA9C9001AB9C300D0E
:10184000300D1124889CC001899C900D900D1124AD
:10185000820F931F0E94680A082F6091290521E0DA
:10186000620F08F46FEFF301EE0FFF1FE85FF44023
:10187000858996890E94C00A7C019401A501632D87
:10188000742D812FEB81FC810995362E472E5394C0
:10189000182FA8CFB0E0A0E0E0E5FCE00C9498356C
:1018A0007C01C0914E018EE0C89FC02D11241EE026
:1018B0001C0F153408F014E40E945E0B882319F005
:1018C000133208F012E20E945E0B811103C0C23293
:1018D00008F4C2E22091290531E0230F08F42FEF2C
:1018E00030E050E040E06FEF7FEF80E090E00E945A
:1018F000F9356901D0E001E02C2FC11740F0812FAC
:101900000E94870BCDB7DEB7E8E00C94B435FE013A
:10191000EA54FD4F808190914F01892309F1409154
:10192000F8044150042E000C550B47FF1BC0C601A4
:1019300060912905600F08F46FEF0E94C00AAC01A6
:10194000609126057091270580912805F70109957A
:101950000E94CA0A462F282F672FCE010E946109D4
:101960002196CACFFA01E850FB4F818982130AC041
:10197000FA01EE0FFF1FE850FB4F818D928D8C1501
:101980009D05B0F241505109D0CFB0E0A0E0EBECA2
:10199000FCE00C9496356C01C0914E018EE0C89F1E
:1019A000C02D11241EE01C0F153408F014E40E9411
:1019B0005E0B882319F0133208F012E20E945E0BCE
:1019C000811103C0C23208F4C2E260912905669514
:1019D00066958091F4049091F5040E94C00AF82E57
:1019E00080E48F0D0E94490A90E8B92EB80E8F2D21
:1019F0000E94490A20E8A22EA80ED0E0C11740F0AC
:101A0000812F0E94870BCDB7DEB7EAE00C94B23588
:101A1000FE01EA54FD4F808190914F018923A1F08E
:101A2000609126057091270580912805EF2C0C2FD9
:101A30002A2D4B2DF60109950E94CA0A462F282F00
:101A4000672FCE010E9461092196D8CFB0E0A0E0B7
:101A5000ECE2FDE00C9492355C01C0914E018EE009
:101A6000C89FC02D11241EE01C0F153408F014E48B
:101A70000E945E0B882319F0133208F012E20E94D4
:101A80005E0B811103C0C23208F4C2E260912905E5
:101A900066958091F4049091F5040E94C00AF82E96
:101AA000D0E0CE01880F991F9C012E503E4F690156
:101AB000C11740F0812F0E94870BCDB7DEB7EEE053
:101AC0000C94AE35FE01EA54FD4F808190914F0198
:101AD000892379F1F60184AD282F2057330B490172
:101AE00085ADE82FE052FF0B3F01889C9001899C57
:101AF000300D300D1124EE9FC001EF9F900D900D21
:101B00001124820F931F0E94680A082F60912605F6
:101B10007091270580912805EF2C9301A401F50110
:101B200009950E94CA0A462F282F672FCE010E94CE
:101B30006109F2E0CF0ED11C2196BACFB0E0A0E04F
:101B4000E4EAFDE00C9497356C01C0914E018EE003
:101B5000C89FC02D11241EE01C0F153408F014E49A
:101B60000E945E0B882319F0133208F012E20E94E3
:101B70005E0B811103C0C23208F4C2E260912905F4
:101B800066958091F4049091F5040E94C00AB82EE5
:101B9000D0E0CE01880F991F9C012E503E4F790155
:101BA000C11740F0812F0E94870BCDB7DEB7E9E067
:101BB0000C94B335FE01EA54FD4F808190914F01A2
:101BC0008923C1F0F70125AD2052330B44AD4057B6
:101BD000550B6091260570912705809128050B2DE6
:101BE000F60109950E94CA0A462F282F672FCE01B9
:101BF0000E946109F2E0EF0EF11C2196D1CFEF9225
:101C0000FF920F931F93CF93DF937C01C0914E01FE
:101C10008EE0C89FC02D11241EE01C0F153408F063
:101C200014E40E945E0B882319F0133208F012E2CC
:101C30000E945E0B811103C0C23208F4C2E26091BF
:101C400029056695669521E0620F08F46FEF809193
:101C5000F4049091F5040E94C00A082FD0E0C11747
:101C600040F0812F0E94870BCDB7DEB7E6E00C94E1
:101C7000B635FE01EA54FD4F808190914F018923D2
:101C800091F0609126057091270580912805202FFD
:101C90004C2FF70109950E94CA0A462F282F672F5B
:101CA000CE010E9461092196DACFB0E0A0E0EBE519
:101CB000FEE00C949635182F80914B01811323C0C0
:101CC00090912505937020914A0130E081E09217B0
:101CD000130609F480E081708093500180912A05F9
:101CE00090914F01981739F080934F0140E060E0E8
:101CF00080E00E946409133288F4E12FF0E0EF5491
:101D0000F94C0C94183681E0E6CF8091500188237D
:101D100089F140E060E080E00E94640980E02AC030
:101D2000C0914E018EE0C89FC02D11240EE00C0F13
:101D3000053408F004E40E945E0B882319F0033296
:101D400008F002E20E945E0B811103C0C23208F467
:101D5000C2E26091260570912705809128050E94B6
:101D6000CA0AF62EE72ED82ED0E0C017D8F0802F62
:101D70000E94870B90914E019F5F90934E018111BD
:101D80000CC082E080934C0180915001811105C00C
:101D9000111103C083E080934C01CDB7DEB7EAE0B8
:101DA0000C94B235FE01EA54FD4F808190914F01B1
:101DB000892331F02D2D4F2D6E2DCE010E9461090A
:101DC0002196D3CFC0914E018EE0C89FC02D112423
:101DD0000EE00C0F053408F004E40E945E0B88232B
:101DE00019F0033208F002E20E945E0B811103C079
:101DF000C23208F4C2E2E0902705F0902805D091A5
:101E000026056D2F7E2D8F2D0E94CA0AD62EC72E35
:101E1000B82E609129056D0F7E2D8F2D0E94CA0A64
:101E2000F62EE72EA82ED0E0C01708F0A0CFFE01B6
:101E3000EA54FD4F908180914F01892359F02A2D5A
:101E40004F2D6E2D90FD03C02B2D4D2D6C2DCE01F1
:101E50000E9461092196E8CFC0914E018EE0C89F93
:101E6000C02D11240EE00C0F053408F004E40E948C
:101E70005E0B882319F0033208F002E20E945E0B29
:101E8000811103C0C23208F4C2E2E0902705D0906D
:101E900028052091290550E4F52E3F2D329F312D44
:101EA0001124F32ED0E0C01708F061CFFE01EA54F0
:101EB000FD4F808190914F018923B9F0FE01EE0F13
:101EC000FF1FEE50FE4F85AD82958F706091260505
:101ED0008F9D600D11247E2D8D2D0E94CA0A462FE4
:101EE000282F672FCE010E9461092196DCCFC09177
:101EF0004E018EE0C89FC02D11240EE00C0F05345A
:101F000008F004E40E945E0B882319F0033208F005
:101F100002E20E945E0B811103C0C23208F4C2E2E9
:101F2000E0902705D09028052091290530E4F32E74
:101F30003F2D329F312D1124F32ED0E0C01708F031
:101F400016CFFE01EA54FD4F808190914F01892305
:101F5000D9F0FE01EE0FFF1FEE50FE4F64ADF69E6E
:101F6000B001112495E0759567959A95E1F78091F8
:101F70002605680F7E2D8D2D0E94CA0A462F282F18
:101F8000672FCE010E9461092196D8CFC0914E01E2
:101F90008EE0C89FC02D11240EE00C0F053408F010
:101FA00004E40E945E0B882319F0033208F002E279
:101FB0000E945E0B811103C0C23208F4C2E2F090AD
:101FC0002605D0912705E0902805609129056695A2
:101FD000669566958091F4049091F5040E94C00A7C
:101FE0000E94490A805887FD8195880F282F3E2D31
:101FF000239F212D1124822F6F2D7D2F0E94CA0A2D
:10200000F62EE72ED82ED0E0C01708F0B0CEFE0195
:10201000EA54FD4F808190914F01892331F02D2D9D
:102020004F2D6E2DCE010E9461092196EDCF88E3E0
:1020300099E00E94FF0D9ECE8EE099E0FACF8BE2F0
:102040009AE00E949E0D96CE8CE09AE0FACF81EF46
:1020500099E00E94260D8ECE85ED99E0FACF8CE0B6
:1020600099E0E7CF83E099E0E4CF8AEF98E0E1CF11
:1020700081EE98E0DECF83ED98E0EBCF88E99AE03F
:10208000E0CF84EC99E0DDCF80EB99E0E2CF86EA07
:1020900098E00E94C50C6ECE88E798E0FACF81E404
:1020A00098E0F7CF8AE398E00E944A0C63CE84E37D
:1020B00098E0FACF8091F80421E0382F321B08F421
:1020C00030E0832F6BE178E00E94970B53CE6BE1F9
:1020D00078E080E0F9CF8091F80421E0382F321BBE
:1020E00008F430E0832F60EE77E0EECF60EE77E02B
:1020F000F0CF8091F80421E0382F321B08F430E053
:10210000832F6EEA77E0E0CF6EEA77E0E2CF80914E
:10211000F80421E0382F321B08F430E0832F66E901
:1021200077E0D2CF66E977E0D4CF8091F80421E060
:10213000382F321B08F430E0832F60E877E0C4CFFB
:1021400060E877E0C6CFF894E82FE295EF70F0E012
:1021500031A1282F2F7081E090E001C0880F2A95CF
:10216000EAF7982F9095932391A392A1892B82A3AC
:10217000789408959091AD0392FF06C0282F28719E
:102180002830F9F4877F846093FF06C0282F2871D8
:102190002831F1F4877E84612091AE0320FF06C0D0
:1021A000382F38713830D9F4877F816021FF06C01D
:1021B000282F28712831D1F4877E816194FD877E94
:1021C0000895282F24712430F9F68B7F8860DCCFA6
:1021D000282F2471243101F78B7E8861DDCF382FC1
:1021E0003171313019F78E7F8860E0CF282F21714F
:1021F000213121F78E7E8861E1CFCF93DF93EC010F
:1022000082389105B1F108F040C08133910509F49D
:102210009DC048F58932910509F48DC08A9709F46B
:102220009CC0C11522E5D20708F0BDC0C11531E53B
:10223000D30708F024C1C83ED10508F0A3C0C13EB1
:10224000D10588F5C83AD10508F08EC0C53AD10548
:1022500008F0F6C0C130D10531F1209721F1C4302A
:10226000D10508F545C08533910509F45FC0C997CC
:10227000C1F68091AD03837009F036C18091AE0341
:1022800083FF11C0C9E2D0E00EC0833E910599F1F1
:1022900070F4803E910501F1823E910511F6809126
:1022A000AD0382FD21C0CE01DF91CF910895863E1E
:1022B000910561F1873E910571F1843E910509F028
:1022C000B0CF8091AE0381FFEECF8091AD03C7EE1A
:1022D000D0E084FD0DC0E7CF8091AD0380FD33C019
:1022E0009091AE0390FFDFCFC3EED0E084FFDBCF51
:1022F000D0E0C0E0D8CF8091AD0382FDF2C09091D4
:10230000AE0390FDF1C084FFCECFF2CF8091AD033C
:1023100083FDDDCFC8CF8091AD0383FDE8C09091F0
:10232000AE0391FFF0CFC4EED0E0BDCF8091AD03FE
:1023300085FFB9CFA7CF8091AD0385FDDBC080912C
:10234000AE0383FFB0CFC9E3D0E0ADCF8091AD0342
:1023500086FFA9CFCAE2D0E0A6CF8091AD0386FF69
:10236000A2CFC1E3D0E09FCFCF3BD10508F6C85A3A
:10237000D0E0CC0FDD1FCA56DE4F0990D881C02DAA
:10238000D46491CFC11540E5D40708F064C0C115ED
:1023900080E4D80708F05CC0CE019A9581159F4172
:1023A00008F481CFA5CFC11536E5D30718F5C115BF
:1023B00045E5D40708F07CC0C11584E5D80708F0CE
:1023C00072C09E01237033279C2F96959695C11558
:1023D000D34508F459C0C1E0D0E002C0CC0FDD1FE6
:1023E0002A95E2F730E2939FC0011124C82BD92B24
:1023F000DA6859CFC1158AE5D80778F4C11529E5FF
:10240000D20708F060C0C11538E5D30708F470CFD3
:10241000DC2FCC27C06FD06A46CFCE0190568115F5
:10242000904208F065CF8D2F8F710E94BA1090E016
:10243000982F882788279F719C012C2BE90141C088
:10244000C55AD0E0CD56DE4FC881D0E0D0642BCF46
:10245000DF70D06A28CFCE018370992721E030E069
:1024600002C0220F331F8A95E2F7C695C69580E217
:10247000C89FE0011124C22BD32BDD6814CFDC2FC1
:10248000CC27C16FD06A0FCFC1E0D0E002C0CC0F23
:10249000DD1F2A95E2F720E2929FC0011124C82B8C
:1024A000D92BDC6800CFDC2FCC27C46FD06AFBCEE1
:1024B0008C2F0E94BA10C82FD0E0DC2FCC27CC275D
:1024C000DF71D062F0CE8C2F8F700E94BA1034E092
:1024D000D695C7953A95E1F7CF709C2FEC01D0695E
:1024E000E2CEC2EED0E0DFCEC0EED0E0DCCEC6EE73
:1024F000D0E0D9CEC5E3D0E0D6CE0E94F90608954B
:1025000080916703811110926703089580959091DF
:102510006603982390936603089580915B039091DE
:102520002A03981301C008958F5F8770FACFA82FF0
:10253000A77023E0969587952A95E1F7FC01EE0FA9
:10254000FF1FE80FF91FE60FF71F50E040E080E0A3
:10255000219130E00A2E02C0369527950A94E2F7C1
:1025600021703327042E01C0220F0A94EAF7822B30
:102570004F5F5F4F4330510559F70895292F9A3027
:1025800068F4863090F490E06CE073E036E0239FCE
:10259000800D911D11240E94971208952C5F223006
:1025A00020F469E073E090E0F6CF80E00895262FF4
:1025B000277091E001C0990F2A95EAF723E07695FC
:1025C00067952A95E1F7FB01EE0FFF1FE60FF71F56
:1025D000E40FF51F50E040E0682F70E08191DF01CB
:1025E00011979B01042E02C0369527950A94E2F7B5
:1025F000217021952827292328272C934F5F5F4F8F
:102600004330510559F70895282F862F9A3070F4DA
:10261000263058F4622F70E026E0929F600D711D05
:1026200011244CE053E00E94D71208959C5F923031
:10263000E0F7622F70E049E053E0F5CF829590E03B
:102640009C01220F331F220F331F2C7C95958795F9
:10265000959587958373282B30E0C901880F991FC2
:102660008A7A359527952575822B08959FB7F8941A
:102670001092DB049FBF9091EA04943009F048C0A7
:102680002091E9002F703091EC00932F917030FD74
:1026900090E8922B25E02093E9002091EB0020FFA9
:1026A00034C02091EE0027FF30C02091DA042223AD
:1026B00021F02091E80025FF28C01092DA0426E0DE
:1026C0003091E80035FF14C08093F1008091E8005C
:1026D00085FD27C08091E80080FFFCCF8091E80055
:1026E0008E778093E8009F709093E90080E00895D2
:1026F0003091EA04343049F43091EB0035FD05C0E7
:10270000215041F481E08093DA049F709093E900B6
:102710008FEF0895EFE9FFE03197F1F700C0000077
:10272000CFCF8FB7F89421E02093DB048FBFDBCFAE
:102730008093D7047093D9046093D8048091EA04FD
:102740008430F9F48093E9008FEF9091E800815094
:1027500095FD06C095ED9A95F1F700008111F5CF32
:102760008091E80085FF0DC050E040E063E070E03C
:1027700087ED94E00E94B1058091E8008E77809308
:10278000E8000895BC0184E00E9498130895BC01FC
:1027900083E00E9498130895CF93DF93EC0181E0CA
:1027A0008093E9008FEF9091E800815095FD06C07D
:1027B00095ED9A95F1F700008111F5CF8091E80031
:1027C00085FF14C050E040E068E070E0CE010E9458
:1027D000B1058091E8008E778093E80088E0FE01E3
:1027E000A0EEB4E001900D928A95E1F7DF91CF91D0
:1027F000089581E08093E00080E28093D8001092F9
:10280000C9008FE19EE40197F1F700C0000087E066
:1028100090EBDC0180932B0590932C05A0932D0564
:10282000B0932E0588E19CE00FB6F894A8958093AC
:1028300060000FBE90936000FFCF6E9A3EB13F7B69
:102840002EB120644FB7F89480E094E0FC015191E0
:10285000CF0168E02EB9000000C057FF3EB9550F08
:10286000000000C000C000C03EB900C06A9591F7EA
:10287000F4E08C3C9F0751F74FBF8FE594E0019740
:10288000F1F700C00000089580917303811110C01A
:102890008091D80080618093D8008AE18A95F1F711
:1028A00000C08091D90080FF0AC081E0809373034B
:1028B00081E090917303913009F080E0089582E007
:1028C000809373030E9461051092EA04F1CF0E9485
:1028D0004414882359F0E091CE04F091CF0430974E
:1028E00029F00190F081E02D0995089580E0089588
:1028F0000F931F930E944414882329F00E94F90625
:102900001F910F9108950E94F90600919D03109167
:102910009E0320919F033091A003600F711F821FBF
:10292000931FEECFCF92DF92EF92FF926B017C016B
:102930000E9444148823A1F02FB7F8946091D30427
:102940007091D4048091D5049091D6042FBF6C1956
:102950007D098E099F09FF90EF90DF90CF90089539
:102960000E947814F4CFCF93DF93C7E2D2E060E007
:10297000CE010E9475362196C11584E0D807B9F7BB
:10298000DF91CF9108950F931F93CF93DF93142F6F
:10299000022F843020F5623010F598E0899FE00125
:1029A000112484E0689FB0011124C60FD71FC95FAE
:1029B000DD4F82E090E0442311F090E080E0632F4F
:1029C0008C0F9D1F0E94753683E090E0112311F05B
:1029D00081E090E0602F8C0F9D1F0E947536DF9183
:1029E000CF911F910F9108951F93CF93DF93122FD3
:1029F0008430E0F46A30D0F44630C0F4C42FD0E024
:102A0000CC0FDD1F9CE0699FC00DD11D112498E7FC
:102A1000899FC00DD11D1124632FCE0187960E947E
:102A20007536612FCE0188960E947536DF91CF9161
:102A30001F910895B0E0A0E0E0E2F5E10C94943538
:102A400081E2E82E86E0F82E01E416E0C0E05801AD
:102A5000D0E015C0F401259134914D2D6D2F8C2FB0
:102A60000E94F41482E0880E911CD39486E0D81260
:102A7000F1CF8CE0A80EB11CDF5FDA3019F0450110
:102A8000D12CE8CF6701D0E0F6012591349141E0E7
:102A90006D2F8C2F0E94C314F6013296259134912C
:102AA00040E06D2F8C2F0E94C31484E0C80ED11C0F
:102AB000D13071F488E0E80EF11CCF5F08581F4F49
:102AC000C43009F0C4CFCDB7DEB7ECE00C94B0351C
:102AD000D1E0DACFCF93C82F6FEF811162E283E2AA
:102AE00090E00E9475366FEFC11163E084E290E0E0
:102AF0000E9475366FEFC11160E185E290E00E949F
:102B00007536CF91089580E00E946A1560E086E2F4
:102B100090E00E9475360E941A150E94B31481E05D
:102B20000E946A150895FF920F931F93CF93DF932E
:102B3000F42E843070F5623060F528E0829F8001C9
:102B4000112434E0639FB0011124060F171F095FA1
:102B50001D4F82E090E0442311F090E080E0800F70
:102B6000911F0E945736C82FD0E0DC2FCC2783E07E
:102B700090E0FF2011F081E090E0800F911F0E9413
:102B800057369E01282BC901CDB7DEB7E5E00C947E
:102B9000B73590E080E0F8CF0F931F93CF93DF938A
:102BA000843030F56A3020F5463010F5C42FD0E07F
:102BB000CC0FDD1F2CE0629FC00DD11D112438E722
:102BC000839FC00DD11D1124CE0187960E945736D8
:102BD000082F10E0102F0027CE0188960E9457364C
:102BE0009801282BC901DF91CF911F910F91089572
:102BF00090E080E0F8CF843070F47A3038F46630BA
:102C000050F4462F672F0E94CC1508957D3F31F474
:102C100041E0623040F090E080E008957C3FD9F7D9
:102C20006230C8F740E00E9493150895CF92DF927A
:102C3000FF920F931F93CF93DF936C0100912405B4
:102C400080916803082BC7E0D0E010E0FC2EC8019B
:102C50000C2E02C0959587950A94E2F780FD0CC072
:102C60002197A0F7F12C8F2DDF91CF911F910F911C
:102C7000FF90DF90CF900895B6018C2F0E94FB1536
:102C80000E94FD10019761F3EECFCF93DF93EC012B
:102C90000E941616BE010E94FB150E94FD10DF91D6
:102CA000CF910895FC0183819481892B29F0808143
:102CB000918189238F3F51F480E00895843FE1F7AB
:102CC00017C0883EA8F0813FB9F712C0808191817A
:102CD0000E94451692959F70963099F358F4925F32
:102CE0009F70923048F7803F19F040F7883E20F7F8
:102CF00081E008959A5FF4CF83E290E00E94573616
:102D0000823289F484E290E00E945736833059F48D
:102D100085E290E00E94573691E0803109F090E022
:102D2000892F8170089580E0FCCFCF9384E090E0FC
:102D30000E945736C82F82E290E00E945736982FA3
:102D40008C2FCF91089546E050E06CE170E085E271
:102D500095E00E9465361092FF0308954F925F92AE
:102D60006F927F928F929F92AF92BF92CF92DF929B
:102D7000EF92FF926091F9037091FA038091FB0347
:102D80009091FC030E9492146B017C010E947814C4
:102D90004B015C018092F9039092FA03A092FB032D
:102DA000B092FC03A091D003E0EDF3E08A2F90E015
:102DB0004FEF5FEF60E070E04C195D096E097F092D
:102DC000A91328C08093D0038091FD03811135C0E1
:102DD00090912505892F837019F0892F8695869506
:102DE00090914C01913009F441C0992341F1923006
:102DF00009F43FC0933009F43FC0FF90EF90DF909B
:102E0000CF90BF90AF909F908F907F906F905F908A
:102E10004F900895218D328D2901712C612C44151C
:102E200055056605770520F481509F5F3296C8CF1F
:102E30002C0D3D1D328F218FF8CF80E0D1CF109225
:102E40004E018092F4049092F504A092F604B092A0
:102E5000F70489E2E0EDF3E0A8EFB4E001900D9211
:102E60008A95E1F781E080934C01C7CF0E94550E0F
:102E7000C4CF0E947307C1CF8091FF0381110E94CC
:102E8000A3166091F4047091F5048091F60490917A
:102E9000F7040E949214603171058105910508F4D0
:102EA000ACCF10924C01A9CF809329059091FF03DC
:102EB000962B9093FF039091FE0390FF16C02FE591
:102EC00031E0662311F021E631E01F928F933F93AA
:102ED0002F9382E096E09F938F930E9458050F9066
:102EE0000F900F900F900F900F900895FC0180812C
:102EF0008730B1F0883011F581818238F9F4809102
:102F00002905873238F08F3538F08E3938F083E074
:102F10008283089580E0FCCF81E0FACF82E0F8CF91
:102F20008181823859F4E2818FE7E43020F4F0E0C7
:102F3000E650FD4F808160E00E9454170895809113
:102F4000290520E1382F321B08F430E0832F61E09F
:102F50000E94541708958091290520E1382F320FDF
:102F600008F43FEF832F61E00E94541708953091D9
:102F70002505337071F18093260560932705413A4A
:102F800008F040EA409328053091FF03322B30933C
:102F9000FF033091FE0330FF1CC050E09927211140
:102FA00019C02FE531E05F934F931F926F939F936A
:102FB0008F933F932F938FED95E09F938F930E9474
:102FC00058058DB79EB70A960FB6F8949EBF0FBEF0
:102FD0008DBF089521E631E0E6CFE5E2F5E04381DB
:102FE00020E1421B08F440E0818121E0628190E011
:102FF0000E94B7170895E5E2F5E0438120E1420F12
:1030000008F44FEF818121E0628190E00E94B717C0
:103010000895E5E2F5E0628120E1621B08F460E0DA
:10302000818121E0438190E00E94B7170895E5E295
:10303000F5E0628120E1620F08F46FEF818121E009
:10304000438190E00E94B7170895E5E2F5E08181A1
:1030500021E0438162818850990B0E94B71708953F
:10306000E5E2F5E0818190E021E04381628108960C
:103070000E94B717089590912505937051F1811121
:1030800029C094609093250510924C018091FF0314
:10309000862B8093FF038091FE0380FF1AC020914E
:1030A0002505269526958FE591E0662311F081E6AA
:1030B00091E01F922F939F938F9385EC95E09F93C0
:1030C0008F930E9458050F900F900F900F900F90C4
:1030D0000F900895833210F09868D4CF880F880F2E
:1030E000982BD0CF8091250586958695815009F43F
:1030F00082E261E00E943B18089580912505869543
:1031000086958F5F833208F081E061E00E943B1872
:1031100008958091FE0380FF08C081EA95E09F93A7
:103120008F930E9458050F900F9085E3809325059B
:103130008091510190915201A091530180932605F5
:1031400090932705A09328058FE7809329058FEF9B
:1031500080932A050E94A3160895B0E0A0E0E3EB57
:10316000F8E10C9493357C015B01842E752E690186
:103170008091740301E010E08A3010F40AE010E05E
:10318000C1E0D0E0B501C701F6010995982E811183
:1031900014C021960C171D07B4F48091FE0380FF24
:1031A0000CC07F928F9284EE92E09F938F930E9447
:1031B00058050F900F900F900F90892DCDB7DEB767
:1031C000EDE00C94AF35CC9F9001CD9F300D300DCC
:1031D000112490E080E045E34A95F1F70000019664
:1031E00028173907C1F7CECFAFE0B0E0EAEFF8E13A
:1031F0000C9493358E010F5F1F4F8AE0D8011D920A
:103200008A95E9F786E3C82E81E0D82EF12CE12CCF
:10321000AA24A394B12C26E3822E21E0922EF6015B
:1032200081916F018F3F09F442C0F894E82FE29535
:10323000EF70F0E021A18F70A50102C0440F551F6F
:103240008A95E2F7CA01922F982B91A392A18095BB
:10325000892382A3789400C0E0E3F1E0712C31E08F
:1032600021912F3F09F46BC0A22FA295AF70B0E05F
:1032700090968C9190E02F7002C0959587952A9535
:10328000E2F780FD5CC0832F782A330F8E169F06ED
:1032900039F7F601319780818F3F11F00E94A3101A
:1032A00050EA5A95F1F7F801EE0DFF1D70828FEF8D
:1032B000E81AF80A95E0E916F10409F0B0CF4AE0FF
:1032C00050E0B80181EA93E00E949936009741F0FE
:1032D0002AE0F801A1EAB3E001900D922A95E1F706
:1032E0000091AC03892B69F181E080936B030E940C
:1032F000050790936A038093690380916903909115
:103300006A030E94EA06059700F110E00A531C4F79
:1033100045E050E061EA73E0C8010E949936C12C93
:10332000892B51F085E0E1EAF3E0D80101900D929C
:103330008A95E1F7CC24C39410926B0307C080E018
:10334000A3CF80916B038111D8CFC12C0E9444146C
:10335000D82EE091AC03DE011B967D01882309F491
:1033600099C085E01D928A95E9F70E2F10E00A5367
:103370001C4FB0907403B9E0BB1508F447C029E0B6
:1033800031E248E651E0B701C8010E94AD18882338
:1033900009F45EC020EF3AE245E751E0B701C80109
:1033A0000E94AD18882309F453C02EE030E24DE7A7
:1033B00051E0B701C8010E94AD18882309F448C044
:1033C0002CEA3FE148E851E0B701C8010E94AD187E
:1033D0008823F1F1F9E0FB1508F453C0109274034F
:1033E0008091AB0390E045E050E0B7018A539C4FD9
:1033F0000E94993621E020937203892BE1F4D12CAD
:103400008D2D8C292F96EDE00C94AF3580916C03B7
:1034100090916D030E94EA06843F914008F0AFCF7F
:1034200080917203882359F385E0D7011D928A9514
:10343000E9F710927203A091AB03B0E0AA53BC4F1E
:1034400085E0FE013B9601900D928A95E1F7D8CF79
:10345000809174038F3F31F08F5F809374038A30C3
:1034600008F4BECF0E94050790936D0380936C0310
:103470008091FE0380FFD4CF8EEA92E00E94BF04C9
:10348000CFCF8091FE0380FFA9CF8BE992E00E940D
:10349000BF04A4CFF0E0EA53FC4F85E0A7E8B3E017
:1034A00001900D928A95E1F765E070E087E893E07E
:1034B0000E945707809386034091C20350E06091B9
:1034C000C10370E063547C4FC7010E94A6368B8510
:1034D00080938D0361E070E0C7010E9457078093DD
:1034E0008C0380908E0390908F03A0909003B090F7
:1034F000910380916E0390916F03A0917003B0913E
:10350000710388169906AA06BB06D1F080926E0355
:1035100090926F03A0927003B09271030E944414C2
:1035200081110EC00E94F906861A970AA80AB90AE4
:1035300080929D0390929E03A0929F03B092A0035D
:1035400086E0E2E9F3E0A5E2B5E001900D928A950C
:10355000E1F710919803112349F08091FD03811147
:1035600005C00E94550E80E00E9473071093FD0372
:1035700047CF0F931F93CF93DF9380916603909172
:103580006503892B8093000390916703992391F041
:10359000892B8093000320E082E093E0FC013191CD
:1035A000CF0131112F5FF3E088309F07B9F7211168
:1035B0000E94801248E050E06DE573E080E093E007
:1035C0000E949936892B09F441C088E0E0E0F3E0DD
:1035D000ADE5B3E001900D928A95E1F7E091CE045C
:1035E000F091CF04309791F10280F381E02D80E0DB
:1035F00093E009958091FE0382FF28C080FF04C0FC
:1036000089E892E00E94BF04D0E0C0E003E812E045
:103610008091FE0380FF0EC0FE01E050FD4F8081CF
:103620001F928F931F930F930E9458050F900F9036
:103630000F900F902196C830D10551F78091FE036D
:1036400080FF04C081E892E00E94BF04DF91CF9127
:103650001F910F91089590E080E00E94410790E053
:1036600080E00E942B07109265030E94B91A08950A
:10367000809324050E942B1B089580912405982F88
:103680009670963021F488600E94381B0895877FD9
:10369000FBCF21E030E001C0220F8A95EAF72095A8
:1036A0008091240582230E94381B089590915C0329
:1036B0008095892380935C03282F277091F4282F0D
:1036C000082E000C330B9217130659F09091AE039D
:1036D00092FF07C08595859585950E94491B10929C
:1036E0005C030895CF93DF93D82FC091AE03C2FB44
:1036F000882780F98D1711F1D0FBC2F9C093AE0372
:103700006091AD0384E090E00E9475366C2F82E2F8
:1037100090E00E94753682E00E94561B8091FE0365
:1037200080FF0CC01F92DF938CE692E09F938F93F3
:103730000E9458050F900F900F900F90DF91CF913E
:10374000089521E030E001C0220F8A95EAF78091C8
:103750002405822B0E94381B0895809368030E94E1
:103760002B1B089510926603E2E0F3E086E0DF0190
:103770001D928A95E9F70E942B1B0895AAE2B0E0FA
:10378000E4ECFBE10C949D358CEE94E02091F1008B
:10379000DC012D93CD01B4E0843F9B07B9F7809104
:1037A000ED04833009F472C0B8F4813009F449C0E3
:1037B000823009F4B3C08091E80083FF91C2809108
:1037C000EC049091ED049A3008F08AC2E92FF0E001
:1037D000EC52F94C0C9418368A3009F48EC08B30B8
:1037E00009F471C0893039F78091EC04813219F7FE
:1037F0008091F0049091F104009711F00297D9F6AE
:103800008091E800877F8093E8008091E80082FF44
:1038100038C09091F3008091F200029731F48091CA
:10382000F100813011F0863021F48091F100809315
:10383000DF048091E8008B778093E8000E94DB052D
:10384000BACF8091EC04813A09F0B5CF8091E800BD
:10385000877F8093E8008091F0049091F104892B98
:1038600061F468E080EE94E070E00E948706809149
:10387000E8008B778093E8009ECF60E090E080E0E6
:10388000F3CF8091EA048111C0CF95CF8091EC04F1
:10389000813A09F090CF8091F0049091F104892B46
:1038A00009F089CF8091E800877F8093E8008091BC
:1038B000E80080FFFCCF80914D018093F100809162
:1038C000E8008E77B9CF8091EC04813209F073CF94
:1038D0008091F0049091F104892B09F06CCF8091D4
:1038E000E800877F8093E8000E94DB058091EE046A
:1038F00080934D010E94B21B5ECF8091EC04813217
:1039000009F059CF8091E800877F8093E8000E94FA
:10391000DB058091EF048093DE044DCF8091EC04B1
:10392000813A09F048CF8091E800877F8093E800D2
:103930008091E80080FFFCCF8091DE04BECF80380C
:1039400099F0823809F0CCC18091F0048F708730F3
:1039500008F0C6C18093E9008091EB0085FB8827C1
:1039600080F91092E90006C08091E8049091E90482
:10397000911182609091E800977F9093E800809386
:10398000F1001092F1008091E8008E77A5C18823A4
:1039900009F493C1823009F0A3C18091EE04811132
:1039A00096C18091F0048F702FEF280F263008F019
:1039B00097C18093E9002091EB0020FF88C19330EC
:1039C00031F48091EB0080628093EB0080C1909194
:1039D000EB0090619093EB0021E030E001C0220FFA
:1039E0008A95EAF72093EA001092EA008091EB00B2
:1039F0008860EACF811174C11091EE041F77809125
:103A0000E3008078812B8093E3008091E800877F3A
:103A10008093E8000E94DB058091E80080FFFCCFE6
:103A20008091E30080688093E30082E0111183E0DD
:103A30008093EA0455C18058823008F051C120912A
:103A4000EE043091EF042C3DE3E03E07A1F583E066
:103A50008A838AE289834FB7F894DE01139620E0C7
:103A60003EE051E2E32FF0E050935700E49120FF55
:103A700003C0E295EF703F5FEF708E2F90E0EA3069
:103A8000C0F0C7968D939D932F5F243159F74FBF98
:103A90008091E800877F8093E8006AE270E0CE01C1
:103AA00001960E9487068091E8008B778093E8005A
:103AB00017C1C096E7CF8091F0049091F104432F95
:103AC00055274330510509F44AC078F54130510576
:103AD00009F47AC08BE790E0E5E3F8E04230510565
:103AE00009F0FEC02091E800277F2093E800209194
:103AF000F2043091F3048217930708F49C0140E02C
:103B00002115310509F065C0411163C08091E800BD
:103B100082FDC9CF8091EA04882329F2853019F209
:103B20008091E80083FFF2CFBECF4132510509F406
:103B30003CC04232510509F0D3C08430910508F0F1
:103B4000CFC0FC01EE0FFF1FEE51FE4F0190F08140
:103B5000E02D82529E4FDC018C9190E01AC03327F9
:103B600021303105D1F02115310561F022303105C8
:103B700009F0B6C0E2ECF8E0E4918E2F90E0E2ECC0
:103B8000F8E007C0EEEEF8E0E4918E2F90E0EEEE64
:103B9000F8E0009709F4A4C0A5CFEEEDF8E0E491B9
:103BA0008E2F90E0EEEDF8E0F4CF8430910508F030
:103BB00097C0880F991FFC01E651FE4F0190F081DC
:103BC000E02D89E090E08ECF82E190E0E0EBF8E03C
:103BD00089CF8091EA04882309F465CF853009F400
:103BE00062CF8091E80083FD5ECF8091E80082FD86
:103BF0008DCF8091E80080FF83CF9091F30080917A
:103C0000F2002115310519F08830910550F041E09E
:103C1000089709F040E08091E8008E778093E800F3
:103C20006FCF44914093F1003196215031090196B4
:103C3000E8CF803809F054C08091E800877F8093F6
:103C4000E8008091EB048093F1009DCE811148C083
:103C50001091EE04123008F043C08091E800877F95
:103C60008093E8001093EB040E94DB05112311F010
:103C700084E005C08091E30087FDFACF81E0809366
:103C8000EA0442E061EC81E00E94FA0542E261EC64
:103C900084E00E94FA0542E261EC82E00E94FA05AB
:103CA00042E260EC83E00E94FA0542E261EC85E0CA
:103CB0000E94FA058091EA0413C08091EE048130DD
:103CC00079F481E0933009F080E08093E904109268
:103CD000E9008091E800877F8093E8000E94DB057F
:103CE0008091E80083FF0AC08091E800877F80937D
:103CF000E8008091EB0080628093EB00AA96E3E0FD
:103D00000C94B9350E94B21B2FEF84E39CE0215044
:103D100080409040E1F700C0000088E19CE00FB6D1
:103D2000F894A895809360000FBE90936000FFCF39
:103D3000882321F00E9486120E94B91A08958823D0
:103D400039F090916603982B909366030E94B91AFC
:103D50000895882391F19CEF980F913A80F4E2E066
:103D6000F3E028E033E09191891303C0DF0111975C
:103D70001C922E173F07B9F70E94B91A089590E2D6
:103D8000980F983050F4877091E001C0990F8A9590
:103D9000EAF7892F0E948612EFCF9BE5980F9330A8
:103DA00028F490E080E00E9441070895885A873106
:103DB00020F490E080E00E942B070895CF93C82F55
:103DC0008823B1F08CEF8C0F813A00F5E2E0F3E04C
:103DD00088E093E0DF012D91C21761F08A179B07FD
:103DE000D1F76C2F80E093E00E9411070E94B91A6E
:103DF000CF9108952191C21303C0DF0111971C9246
:103E00008E179F07B9F70E94B91AEBCF80E28C0F8B
:103E1000883068F4C77021E030E001C0220FCA95F5
:103E2000EAF780916603822B80936603DFCFEBE590
:103E3000EC0FE33040F4F0E0ED56FE4F808190E06F
:103E40000E944107D5CFC85AC73190F6EC2FF0E059
:103E5000EE0FFF1FEA56FE4F808191810E942B07D3
:103E6000C7CF1F93CF93DF93182FD0E0C0E08933E3
:103E700011F4C0E5D0E0812F0E94DE1E209739F4B6
